:1000000061C100007CC100007AC1000078C100001D
:1000100076C1000074C1000072C1000070C1000010
:100020006EC100006CC100006AC10000E8C500009C
:1000300066C1000064C1000062C100000C94730935
:100040005EC100005CC100005AC1000003C2000094
:1000500056C1000054C1000052C1000050C1000050
:100060004EC100004CC100004AC1000048C1000060
:1000700046C100001F0F350F3A0F3F0F480F4F0FBB
:10008000540F5E0F640F6B0F710F760F7E0F2004FD
:100090002B04310437043F0444044B048A04A604AF
:1000A000BC04C604D204E6049D07C0075109C0077A
:1000B000510907082908510914092709240C290C9A
:1000C000360C410C500C580C940C070D070DA40C69
:1000D000B50CC90CD40CE00CEF0C05010980A10192
:1000E0008501198129831500250195037501810278
:1000F000950175058101C0050C0901A10185020961
:10010000B009B109B209B309B409B509B609B7090B
:10011000B809CD09E209E909EA0A8A010A92010A45
:1001200094010A21020A23020A24020A25020A274C
:10013000020A2A0215002501951675018102950112
:1001400075028101C005010906A1010508190129EF
:10015000031500250195037501910295017505911F
:1001600001050719E029E7150025019508750181AA
:100170000205071900293115002501953275018105
:100180000295017501810105071933299B15002589
:1001900001956975018102950175018101050719B4
:1001A0009D29A41500250195087501810295017509
:1001B000038101C00600FF0901A101090215002504
:1001C000FF7508950881020903150025FF7508953C
:1001D000089102C005010906A10175019508810178
:1001E00095017508810195057501910195017503CA
:1001F0009101950675088101C009026D0004010096
:10020000A0320904000001030101000921110100CD
:10021000012225000705810308000A0904010001E5
:1002200003000000092111010001222000070583BD
:100230000308000509040200010300000009211160
:10024000010001226F000705820320000A09040350
:10025000000103000000092111010001226B0007C9
:1002600005840308000A1201100100000020810427
:1002700002000100010200012203690062006D001A
:100280002D00630061007000730065006E00730054
:1002900065002D0075007300620000002203540009
:1002A0006F006D00200057006F006E0067002D008A
:1002B00043006F0072006E0061006C006C00000073
:1002C0000403090411241FBECFEFD4E0DEBFCDBF6D
:1002D00011E0A0E0B1E0E6E2F1E202C005900D928B
:1002E000A636B107D9F713E0A6E6B1E001C01D922A
:1002F000AE32B107E1F70E947B0D0C94911080CED5
:1003000083B185FB882780F991E089270895909132
:100310001C039623811102C031F402C0992319F005
:1003200010924B021CC080914B0291E0980F909369
:100330004B02811114C0E42FE695E695E695F0E0B6
:10034000E25DFD4F477081E090E0042E01C0880F10
:100350000A94EAF79081892B808381E0089580E0F8
:100360000895EF92FF920F931F93CF93DF938C0129
:1003700091E0EE24E394F12C461720F120E030E0E8
:10038000A62FB0E0AA0FBB1FAA0FBB1FE801C90F21
:10039000D11DFD01E20FF31FE35BFD4F8081833030
:1003A0004CF08881F701022E01C0EE0F0A94EAF7A3
:1003B000E82BE8832F5F3F4F2430310551F76F5F03
:1003C0009F5FDACFDF91CF911F910F91FF90EF9058
:1003D0000895AF92BF92DF92EF92FF920F931F9317
:1003E000CF93DF93D82EEFEFE80FE33040F4F0E047
:1003F000EE0FFF1FE75AFE4FA080B18003C082E0DE
:10040000A82EB12C00E010E0C0E0D0E07E01E00EAC
:10041000F11EC5018E0D9F1D0E9468108F3F09F4CB
:1004200080E0F701E055FD4F80832196C430D1056F
:1004300069F70C5F1F4F0C35110531F7D0920C0393
:10044000DF91CF911F910F91FF90EF90DF90BF90C0
:10045000AF9008951F920F920FB60F9211248F93B1
:100460009F934698449A459A4598449880E0909185
:10047000A902891720F4459A45988F5FF8CF469ACC
:1004800082E0809381009F918F910F900FBE0F901B
:100490001F901895EEE6F0E080818D7F8083EFE677
:1004A000F0E080818D7F808315BC109281008CE507
:1004B000EDE4F2E0DF011D928A95E9F7089584B535
:1004C000826084BD89E187BDEEE6F0E080818260D4
:1004D000808385B5836085BD1092800088E090E0C0
:1004E0009093890080938800EFE6F0E0808182603D
:1004F0008083089524982598269827982C982D98DD
:100500002E982F981092AB021092AA028091170396
:10051000823019F4249A259A269A0895EBDF809167
:100520001703813029F038F083508C3020F42D9A55
:10053000269A279A2F9A08959093AF028093AE023D
:100540002898880F991F880F991F9EBD0DB407FE2C
:10055000FDCF9EB58EBD0DB407FEFDCF8EB5289A9A
:100560000895AF92BF92CF92DF92EF92FF920F93D6
:100570001F93CF93DF93B0900C0380E02ADF40EB12
:1005800052E080E0A12CD12CE82FE695E695E69587
:10059000F0E0E85EFC4F208130E0982F977002C0B9
:1005A000359527959A95E2F720FD12C020E030E0BE
:1005B000FA01E20FF31F9081992329F0913011F491
:1005C000A39401C0D3942F5F3F4F2430310581F7AE
:1005D0008F5F4C5F5F4F8731B9F6C0E0D0E0EE240B
:1005E000EA9493E0F92E00E010E0C701801B910B24
:1005F0008230910508F44BC0EC01D695C795C00F29
:10060000D11FCE0199DF10924C0280914C028431AF
:10061000E0F340EB52E020E030E0A0E0E22FE6958E
:10062000E695E695F0E0E85EFC4F808190E0622F71
:10063000677002C0959587956A95E2F780FD1AC0AC
:1006400080E090E0B901660F771F660F771FFB010E
:10065000E80FF91FE35BFD4FE081E3303CF4FA0162
:10066000E80FF91FE081E23008F0AF5F01968430B7
:10067000910569F72F5F3F4F4C5F5F4F2731310581
:1006800069F6AD1510F08E01B0CF7E01AECF8E01B0
:10069000CC24CA94A3E0DA2EE12CF12CC6018E19E9
:1006A0009F098230910508F44BC0EC01D695C7959F
:1006B000CE0DDF1DCE0140DF10924C0280914C0226
:1006C0008431E0F380EB92E020E030E0A0E0E22F24
:1006D000E695E695E695F0E0E85EFC4F408150E057
:1006E000622F677002C0559547956A95E2F740FD05
:1006F0001BC040E050E0B901660F771F660F771FFF
:10070000FB01E40FF51FE35BFD4FE081E3303CF0BC
:10071000FC01E40FF51FE081E13009F4AF5F4F5FAA
:100720005F4F4430510561F72F5F3F4F04962731EB
:10073000310569F6AA1510F06E01B0CF7E01AECF7B
:10074000C8018C1B9D0B63E070E00E942110CB015F
:100750008C0F9D1FF1DEE2DE8B2DDF91CF911F917B
:100760000F91FF90EF90DF90CF90BF90AF9031CE80
:10077000EF92FF920F931F93CF93DF93E901D8017C
:1007800021E08533920709F040C08091030188235E
:1007900009F425C11092030190913E0191111FC1EE
:1007A0003EE2E32E32E0F32E60E0F70120812223C7
:1007B00001F120E030E07CEF790FF701408150E05B
:1007C000022E02C0559547950A94E2F740FF0CC0EF
:1007D000192F120F472F420F413A30F4AE01460F46
:1007E000511DFA0112836F5F2F5F3F4F2830310593
:1007F00021F7FFEFEF1AFF0A985F983AB1F6909150
:100800004A02988328E030E014C121E08532920743
:1008100009F0E7C020913E0188E0FE0111928A951F
:10082000E9F7E0911B03E8838E2F90E0FC013197FC
:10083000ED30F10508F0CEC0E95BFF4F0C943510A8
:1008400084E0898398E09A8397E19B838C8381E09D
:100850008D832E83A4C046E060E0CE0182DD83E07C
:100860000BC04DE067E0CE017CDD84E005C044E1D3
:100870006EE0CE0176DD85E080931B03ABC047E1DF
:1008800065E1CE016EDD8BC09091AE028091AF022A
:1008900099838A8384C0E0900C03F0906701FE1472
:1008A00011F08F2D96DD909166018F2D8295880F26
:1008B000880F807C892B89832296692F70E0660FD0
:1008C000771F660F771F40E050E0FA01E60FF71F31
:1008D000E055FD4F808189934F5F5F4F4430510554
:1008E000A1F79F5F973119F0909366010BC01092AA
:1008F000660191E09F0D943019F09093670102C05A
:1009000010926701809167018E1509F463C08E2DE6
:1009100060DD60C0809168018983E82FF0E0EE0F10
:10092000FF1FEE0FFF1FE35FFC4F4081518162818B
:1009300073814A835B836C837D838F5F823019F080
:100940008093680147C01092680144C0EFE5F1E070
:1009500080E090E022E0280F31910196DE01A80F9F
:10096000B91F3C93332321F08630910599F727E096
:10097000C20FD11D188213C0809117038983809103
:1009800016038A83809115038B8309C08091180315
:1009900090911903A0911A0389839A83AB831092D3
:1009A0001B0318C060916901698370E0660F771FAF
:1009B000660F771F44E050E0CE0102960E94581067
:1009C000809169018F5F8093690104C019828091D1
:1009D0004C028A8388E090E0F8019183808380E074
:1009E00081C0F1E085319F0739F5809104018823AA
:1009F000B1F31092040180913E01882381F39E019E
:100A00002F5F3F4F6EE272E095E1960FFB0141913F
:100A1000BF01F90141939F019613F8CF9981987F07
:100A200099839D899F719D8B90914A02988326E1BD
:100A300030E02D933C9356C08550914081F6FB01E8
:100A40008081882319F08093000104C08091000107
:100A5000FB018083809100018130D9F480910201F3
:100A6000882309F4BCCF1092020190914202929522
:100A700096959770988320916A01291719F09093A1
:100A80006A0101C080E021E030E02D933C9392E0C8
:100A900027C0823009F0A3CF80910101882309F497
:100AA0009ECF10920101809143028883809144027D
:100AB0008983809145028F738A83EBE6F1E080E0C1
:100AC00023E02E0F99913081391711F0908381E046
:100AD00031962E13F7CF23E030E02D933C9391E035
:100AE00090930001DF91CF911F910F91FF90EF90B4
:100AF00008952091E4003091E50095E64091EC00E6
:100B0000842F817040FF22C08091E80080FD1CC0CE
:100B100080912503882391F0853091F08091EB003E
:100B200085FD10C04091E4005091E5004217530745
:100B300029F39A01915011F784E0089582E0089515
:100B400083E0089581E0089580E008954091E800F1
:100B500042FFDECF089580911D0387FF11C0809171
:100B6000E80082FD05C0809125038111F8CF11C0F6
:100B70008091E8008B770BC080912503882349F092
:100B80008091E80080FFF8CF8091E8008E77809315
:100B9000E8000895982F953058F59093E90098173C
:100BA00039F07091EC002091ED005091F00003C0FD
:100BB000242F762F50E021FF19C03091EB003E7FAB
:100BC0003093EB003091ED003D7F3093ED0030919C
:100BD000EB0031603093EB007093EC002093ED005C
:100BE0005093F0002091EE0027FF07C09F5FD3CF06
:100BF0008F708093E90081E0089580E008951F924E
:100C00000F920FB60F9211242F933F934F935F9340
:100C10006F937F938F939F93AF93BF93EF93FF93C4
:100C20008091E10082FF61C08091E20082FF5DC09F
:100C30008091E1008B7F8093E1008091430190914E
:100C40004401009729F00197909344018093430158
:100C50008091330190913401009729F0019790938E
:100C600034018093330180912301909124010097F6
:100C700029F001979093240180932301809113011F
:100C800090911401009729F001979093140180939B
:100C900013018091AB028F3F19F08F5F8093AB02FD
:100CA00080911703813021F000F183508C30E8F4FB
:100CB0009091AB0280911603981302C02E9815C034
:100CC00020911503921303C083E085BD0EC080916F
:100CD000AA02882351F0291740F41092AB028150E8
:100CE0008093AA022E9A15BC16BC8091E10080FF69
:100CF00017C08091E20080FF13C08091E2008E7FD8
:100D00008093E2008091E20080618093E200809114
:100D1000D80080628093D80019BC10922503EADBCA
:100D20008091E10084FF2DC08091E20084FF29C002
:100D300084E089BD86E089BD09B400FEFDCF8091C5
:100D4000D8008F7D8093D8008091E1008F7E8093C2
:100D5000E1008091E2008F7E8093E2008091E200CA
:100D600081608093E2008091AD02811106C0809184
:100D7000E30087FD02C081E001C084E08093250389
:100D8000CDDB8091E10083FF24C08091E20083FFEE
:100D900020C08091E100877F8093E10082E0809312
:100DA00025031092AD028091E1008E7F8093E100D7
:100DB0008091E2008E7F8093E2008091E20080616A
:100DC0008093E20042E260E080E0E4DE81E0809334
:100DD0003E01FF91EF91BF91AF919F918F917F91D4
:100DE0006F915F914F913F912F910F900FBE0F9098
:100DF0001F9018952091230330912403261737075D
:100E000048F06115710539F42091E8002E772093A0
:100E1000E80001C0B90140E06115710581F1209140
:100E200025032223E9F12530E9F12091E80023FD93
:100E300035C02091E80022FD2BC02091E80020FF62
:100E4000EBCF2091F20030E0FC01CF01611571057C
:100E500059F02032310540F481918093F1006150C6
:100E600071092F5F3F4FF1CF41E02032310509F08A
:100E700040E02091E8002E772093E800CDCF41118B
:100E8000CECF06C080912503882351F0853051F0E4
:100E90008091E80082FFF6CF80E0089581E0089518
:100EA00082E0089583E008950F931F93CF93DF931B
:100EB000CDB7DEB7AA970FB6F894DEBF0FBECDBF91
:100EC00080912503882309F403C21091E9001F7063
:100ED0009091EC00892F817090FD80E8182B109282
:100EE000E9008091E80083FFEAC1EDE1F3E088E0EA
:100EF0008E0F9091F10091938E13FBCF85E391E0DB
:100F0000A6D385E291E0A3D385E191E0A0D385E06B
:100F100091E09DD38091E80083FFC3C180911D03C0
:100F200090911E03492F50E04A30510508F0B9C195
:100F3000FA01EC5AFF4F0C943510803881F082385A
:100F400009F0AFC1809121038F708093E9008091F7
:100F5000EB0085FB882780F91092E90007C080919B
:100F6000AC02882311F082E001C080E09091E8009B
:100F7000977F9093E8008093F1001092F10060C198
:100F8000282F2D7F09F08DC1882319F0823061F060
:100F900088C180911F03813009F083C1933009F02B
:100FA00080E08093AC022DC080911F03811129C085
:100FB000809121038F7009F474C18093E9009091AE
:100FC000EB0090FF1EC090911E03933021F480919E
:100FD000EB00806214C09091EB0090619093EB0065
:100FE00021E030E0A90102C0440F551F8A95E2F7C5
:100FF0004093EA001092EA008091EB0088608093B1
:10100000EB001092E9008091E800877F1CC18111FC
:1010100048C100911F030F778091E3008078802BF7
:101020008093E3008091E800877F8093E80093DD60
:101030008091E80080FFFCCF8091E300806880937E
:10104000E300011102C082E001C083E08093250328
:1010500028C18058823008F024C180911F039091EC
:1010600020038C3D53E0950771F583E08A838AE283
:1010700089834FB7F894DE01139620E03EE051E2F9
:10108000E32FF0E050935700E49120FF03C0E29576
:10109000EF703F5FEF708E2F90E0EA3010F0C79650
:1010A00001C0C0968D939D932F5F243149F74FBFA8
:1010B0008091E800877F8093E8006AE270E0CE01CB
:1010C000019698DEABC0E0912103292F332723300E
:1010D0003105A9F06CF42130310509F4F4C0223057
:1010E000310509F0DEC08DE690E0E9EFF1E04CC09B
:1010F0002132310531F12232310589F1D2C09927EF
:101100008130910571F08230910599F0892B09F0B9
:10111000C8C0E0ECF2E0E4918E2F90E0E0ECF2E069
:1011200030C0ECE9F2E0E4918E2F90E0ECE9F2E0DF
:1011300028C0E8E7F2E0E4918E2F90E0E8E7F2E0E3
:1011400020C0E43008F0ADC0F0E0EE0FFF1FEF5A12
:10115000FE4F0190F081E02D89E090E015C0E43071
:1011600008F09FC08E2F90E0FC01EE0FFF1FE75BA1
:10117000FE4F0190F081E02DDC01AB5BBE4F8C9106
:1011800090E0009709F48DC02091E800277F20931C
:10119000E80020912303309124032817390708F42D
:1011A000C90140E0009769F1209125032223B1F1A4
:1011B0002530A1F12091E80023FD30C02091E80006
:1011C00022FD28C02091E80020FFECCF2091F20002
:1011D00030E0009759F02032310540F444914093BB
:1011E000F100319601972F5F3F4FF3CF41E020325E
:1011F000310509F040E02091E8002E772093E800C7
:10120000D1CF4111D1CF06C080912503882331F081
:10121000853021F08091E80082FFF6CF8091E800D0
:101220008B778093E8003DC0803809F03AC0809108
:10123000E800877F8093E8008091AD028093F10001
:101240008091E8008E778093E80085DC2AC08111C8
:1012500028C000911F03023020F58091E800877FAD
:101260008093E8000093AD0276DC011106C0809106
:10127000E30087FD02C081E001C084E08093250384
:1012800085E391E0A6D185E291E0A3D185E191E0EB
:10129000A0D185E091E09DD18091E20084608093AF
:1012A000E2008091E80083FF0AC08091E800877F18
:1012B0008093E8008091EB0080628093EB001F70C8
:1012C0001093E90005C082E190E0E6E6F2E05CCF31
:1012D000AA960FB6F894DEBF0FBECDBFDF91CF91B7
:1012E0001F910F9108951F920F920FB60F92112424
:1012F0002F933F934F935F938F939F93AF93BF939E
:10130000EF93FF93CF93DF9300D000D0CDB7DEB73C
:1013100019821A821B821C828091A902873118F0DF
:10132000469888E137C0489B02C091E09983499B69
:1013300002C091E09A834A9B02C091E09B834B9B41
:1013400002C091E09C83DE01119620E030E090E045
:10135000880F991F880F991F57E04D91FC01E20FEC
:10136000F31FE35BFD4F442341F040814150408334
:10137000408143304CF4108207C040814F5F40836E
:10138000408143300CF050832F5F3F4F24303105B4
:1013900021F7C6CF459A45988150E1F7469A80914A
:1013A000A90297E18F5F873130F080914C028F5F07
:1013B00080934C0280E0E82FE695E695E695F0E014
:1013C000E85EFC4F208130E0482F477002C0359521
:1013D00027954A95E2F720FF03C0915019F787E15E
:1013E0008093A902109281001092850010928400CF
:1013F0000F900F900F900F90DF91CF91FF91EF9191
:10140000BF91AF919F918F915F914F913F912F919C
:101410000F900FBE0F901F9018952F923F924F92F2
:101420005F926F927F928F929F92AF92BF92CF9274
:10143000DF92EF92FF920F931F93CF93DF9300D031
:101440001F92CDB7DEB77C014DB65EB68091250305
:10145000843009F0A3C08091E4009091E500F70189
:10146000228533852817390709F498C081818F7048
:101470008093E9008091E80085FF90C08DB69EB60C
:10148000408550E08DB79EB7841B950B0FB6F8943E
:101490009EBF0FBE8DBFEDB7FEB731966F015F01E6
:1014A0001B821A82198260E070E0CF01FAD58E01AA
:1014B0000F5F1F4F960140E0BE016D5F7F4FC70178
:1014C00057D9282EF70184859585892B51F091E015
:1014D00080E026853785232B09F090E0092F182F0F
:1014E00002C000E010E0F7016680778061147104AB
:1014F00089F049815A81B301C601BDD533243394A3
:10150000892B09F4312CF701408550E0B601C30165
:10151000BFD501C0312C89819A81892B99F1211085
:1015200004C0311002C0012B69F1F7018485958553
:101530009787868781818F708093E9008B818111E5
:101540008093F10009811A81D4DA882369F08091AF
:10155000E8008E778093E80015C0F50181915F0166
:101560008093F100015011090115110581F380915B
:10157000E80085FDF2CF8091E8008E778093E80047
:1015800093DCE2CF8091E4009091E500F70193872E
:1015900082870FB6F8949EBE0FBE8DBE0FB6F8942C
:1015A0005EBE0FBE4DBE0F900F900F90DF91CF919A
:1015B0001F910F91FF90EF90DF90CF90BF90AF9071
:1015C0009F908F907F906F905F904F903F902F9063
:1015D0000895CF93DF93FC01DC01199687E0ED01BC
:1015E00019928A95E9F781E0818784EF91E09587E8
:1015F000848783E084836181611102C081E024C01B
:1016000095810280F381E02D862F8F70853010F058
:1016100080E01AC0923010F442E001C046E028E0B9
:1016200030E090E02E173F0720F49F5F220F331F1A
:10163000F9CF9295907F492B661F6627661F606CD5
:10164000A9DA8111DBCFE4CFDF91CF9108958F929A
:101650009F92AF92BF92CF92DF92EF92FF920F9341
:101660001F93CF93DF9300D01F92CDB7DEB76C01ED
:10167000EDB6FEB68091E80083FF28C2F6018081B6
:1016800090E020912103309122032817390709F0B7
:101690001DC280911E03833009F4BFC130F4813034
:1016A00071F0823009F4F6C111C28A3009F4DAC14E
:1016B0008B3009F4C3C1893009F008C24DC0809154
:1016C0001D03813A09F002C28DB69EB61A821982B4
:1016D00080911F03109120038B83F6018085482F92
:1016E00050E08DB79EB7841B950B0FB6F8949EBF44
:1016F0000FBE8DBFEDB7FEB731965F0160E070E0C1
:10170000CF01CFD44FEF410F8E010F5F1F4F9501D7
:10171000BE016D5F7F4FC6012BD8F6018681978190
:10172000009721F0408550E0B501B2D41092E90055
:101730008091E800877F8093E80069817A81C50104
:1017400059DB8091E8008B778093E8000FB6F8941E
:101750009EBE0FBE8DBEBAC180911D03813209F0BD
:10176000B5C10DB71EB740912303509124033091AA
:101770001F038DB79EB7841B950B0FB6F8949EBFC1
:101780000FBE8DBF01962091E800277F2093E800CF
:101790004115510529F42091E8002B772093E800AA
:1017A000FC014115510521F120912503222321F14E
:1017B000253011F12091E80023FD1EC02091E800A2
:1017C00022FFEFCF2091F200222331F02091F1008F
:1017D000219341505109B1F72091E8002B772093D4
:1017E000E800DFCF20912503222331F0253021F0BE
:1017F0002091E80020FFF6CF2091E8002E7720937B
:10180000E800A1E0B0E0311102C0A0E0B0E0E5E303
:10181000CE16E1E0DE0629F420913E012111F7C049
:10182000F1C0F5E2CF16F1E0DF0609F0E2C0A80F43
:10183000B91FEC914E2F50E04F30510508F0E7C032
:10184000FA01E25AFF4F11C411968C9180931B0349
:10185000DEC011962C91119712968C9190E0982FE2
:101860008827820F911D0E949C02D1C011968C91F5
:10187000882309F4CCC00E944A02E0E0F8E109950F
:10188000C6C011968C91882309F4C1C06091AE0244
:1018900080E090E034D46091AF0281E090E09DC0A0
:1018A00011968C91882309F4B2C00E94B102AFC096
:1018B00013966C91139712962C91129711969C91F6
:1018C000492F4F739295969596959370473108F0EE
:1018D0009EC0243008F09BC0EFEFE90FE33040F4E6
:1018E000F0E0EE0FFF1FE75AFE4FA081B18102C06A
:1018F000A2E0B0E080910C0330E050E098130AC001
:10190000FA01EE0FFF1FEE0FFF1FE20FF31FE0556E
:10191000FD4F6083CA01880F991F880F991F820F9E
:10192000931F8A0F9B1F59C012966C9112971196A4
:101930008C91883008F06BC090E0FC01E35FFC4FB5
:1019400060838E589E4F49C013968C9113971296C0
:101950009C91129711962C91209317039093160344
:10196000809315030E948E0252C011968C91882399
:1019700009F44DC0609117038AE791E0C0D36091EC
:1019800016038BE791E0BBD3609115038CE791E0E0
:1019900024C011968D919D91AC91809318039093E2
:1019A0001903A0931A0333C011968C91882379F1FF
:1019B00043E050E06DE771E088E193E091D327C008
:1019C00012968C91129790E0982F882711962C915F
:1019D000119713966C91820F911D91D318C0119697
:1019E0008C91882319F00E945F0211C00E944A0264
:1019F0000EC0F5E1CF16F1E0DF0649F420913E017B
:101A0000222329F0A80FB91F8C9180931C030FB6D5
:101A1000F8941EBF0FBE0DBF59C080911D03813ABF
:101A200009F054C08091E800877F8093E80080919E
:101A3000E80080FFFCCFF601818540C080911D0346
:101A4000813209F043C08091E800877F8093E800ED
:101A500082D890911F0381E0911101C080E0F601CE
:101A6000818734C080911D03813281F58091E80027
:101A7000877F8093E8006FD880911F0390912003A7
:101A8000882736E0969587953A95E1F7F601958790
:101A900084871CC080911D03813AC1F48091E800C5
:101AA000877F8093E8008091E80080FFFCCFF601FB
:101AB0008485958596958795969587958093F10071
:101AC0008091E8008E778093E80045D80FB6F894AF
:101AD000FEBE0FBEEDBE0F900F900F90DF91CF9125
:101AE0001F910F91FF90EF90DF90CF90BF90AF903C
:101AF0009F908F90089584B7877F84BF88E10FB649
:101B0000F89480936000109260000FBE90E080E82F
:101B10000FB6F89480936100909361000FBE219AF4
:101B2000209A229A84E58CBD8DB581608DBD289A5E
:101B30003C9A3D9A3E9A88E1459A45988150E1F752
:101B4000469A809163008E7F8093630081E080934A
:101B50006E011092E2001092E1008091D8008F7720
:101B60008093D8008091D80080688093D8008091BD
:101B7000D8008F7D8093D80084E089BD86E089BD40
:101B800009B400FEFDCF109225031092AD02109211
:101B9000AC0242E260E080E00E94CA058091E10070
:101BA0008E7F8093E1008091E20081608093E2006B
:101BB0008091E20088608093E2008091E0008E7F57
:101BC0008093E000789443E050E06DE771E088E1B5
:101BD00093E06ED2809118038F3F71F480911903C6
:101BE0008F3F51F480911A038F3F31F41092180304
:101BF0001092190310921A038CE5EDE4F2E0DF0174
:101C00001D928A95E9F710922D0280E00E94E90169
:101C100048E050E062E771E08DE093E049D28FEF59
:101C200080930F022FE6E22E21E0F22E00E010E07A
:101C3000CFE7D2E035E0B32EF7012B2D11922A9594
:101C4000E9F7CE0106968115944080F5CE0140D289
:101C50009FEF980F9E3F50F5D7011496DC93CE93DB
:101C600013978C93CE01019633D2F801E159FE4FC0
:101C70004F0181836E01F3E0CF0ED11CCE0102969D
:101C800027D2D40112968C93C60122D2C82FD0E05D
:101C9000CC0FDD1F2196CC0DDD1DCE0119D2282FD2
:101CA00030E0220F331FC20FD31F02C0C0E0D4E0C8
:101CB000B5E0EB0EF11C0B5F1F4F003A110509F068
:101CC000BBCF8AE791E004D2C82F8F3008F0C0E084
:101CD0008CE791E0FDD1D82F8BE791E0F9D1C0934B
:101CE000170380931603D0931503CFE1DEE4219709
:101CF000F1F700C000000E945F0281E090E0E8D1AF
:101D0000C82FD0E0DC2FCC2780E090E0E1D1FE01AD
:101D1000E82BCF010E949C028091AE029091AF020D
:101D2000019611F40E94B1028EE292E01DE1180FBB
:101D3000CC24C394D12C80E192E00DE1080F8DE01A
:101D400093E0A8E0FA2EF80E80913E01882319F066
:101D50008091040102C08091030181110DC1A0E1B5
:101D6000B2E04EE252E0FA01CD012081EC0129936C
:101D7000CE0111921E13F9CF60E070E020E030E058
:101D8000C901880F991F880F991F860F971FFC01A3
:101D9000E35BFD4FE081E330C4F0FC01E055FD4F13
:101DA0008081883E90F4E82FE695E695E695F0E090
:101DB000E25DFD4F8770E60102C0CC0FDD1F8A9502
:101DC000E2F7CE019081892B80832F5F3F4F27312F
:101DD0003105B1F66F5F7F4F6430710579F68EE2A1
:101DE00092E0E0E1F2E03191EC012991CE01321371
:101DF00004C00E13F8CFE12C15C080911703813079
:101E000009F008C13091AA0220E09D91FA01819168
:101E1000AF01981307C12F5F2A31B9F73093AA0297
:101E2000EE24E394E09117038E2F90E0FC013297AB
:101E3000ED30F10508F073C0E65CFF4F16C18091EC
:101E40001C0380FF02C02D9A01C02D9880911C03B5
:101E500081FF02C02E9A01C02E9880911C0382FF40
:101E600002C02C9A5CC02C985AC00E94800149E3A1
:101E700062E009C00E94800149E362E00DC00E9457
:101E8000800143E561E00E948701EE20E1F13DC061
:101E90000E94800143E561E091E08927F4CF0E9430
:101EA0008001811105C03BC00E948001811137C0B3
:101EB00080914A02826080934A0231C00E94800170
:101EC000882331F081E017C00E9480018823D1F37C
:101ED00010922D0224C00E9480018823C9F382E061
:101EE0000AC00E9480018111F3CFF9CF0E948001C6
:101EF000882371F383E080932D0211C00E9480013A
:101F00008111E6CFF7CF882361F081E08093030150
:101F100080930401809302018093010102C0E110CB
:101F2000F4CF8091490280FF03C010922D020DC0B2
:101F300081FF02C081E007C082FF02C082E003C0CF
:101F400083FF03C083E080932D0280912D02909146
:101F50004802977061F0EDE0F3E02191322F329565
:101F60003F70391302C0822F8F70FE12F6CF90910E
:101F70000C0389130E94E90180912503882321F035
:101F8000809125038530B9F58091AC02882399F1C1
:101F9000EEE2F2E020E041914423A1F080E090E005
:101FA00050E0BA01082E02C0759567950A94E2F7D1
:101FB00060FF04C0322F380F343040F4019688306F
:101FC000910579F7285F283E31F715C084E089BD77
:101FD00086E089BD09B400FEFDCF8091D8008F7DD9
:101FE0008093D8008091E00082608093E00080912F
:101FF000E00081FDFCCF85E391E00FDA85E291E01E
:102000000CDA85E191E009DA85E091E006DA0E94D8
:1020100054079ACE813008F403CF83508C3008F0F7
:10202000FFCEF0CE892B8927211101C0807F91E05E
:10203000930F882309F4EFCE3FEF380F8323392F16
:10204000F6CFAA1BBB1B51E107C0AA1FBB1FA617D7
:10205000B70710F0A61BB70B881F991F5A95A9F751
:1020600080959095BC01CD010895EE0FFF1F05905E
:10207000F491E02D0994FB01DC0104C08D910190E5
:10208000801921F441505040C8F7881B990B0895DE
:10209000FB01DC0102C001900D9241505040D8F785
:1020A0000895DC0101C06D9341505040E0F7089560
:1020B000DC01CB01FC01F999FECF06C0F2BDE1BD08
:1020C000F89A319600B40D9241505040B8F70895F7
:1020D000F999FECF92BD81BDF89A992780B50895F0
:1020E000DC01A40FB51F4150504040F0CB01840FDC
:1020F000951F2E9105D041505040D8F70895262FB6
:10210000F999FECF92BD81BDF89A019700B40216ED
:1021100039F01FBA20BD0FB6F894FA9AF99A0FBE9B
:062120000895F894FFCFC2
:102126000101010101038408000001000003000011
:1021360000000000000282200000010000160000DE
:1021460000000000000183080000012603080000CB
:1021560000000000000081080000010000080000E7
:10216600000000000025206F6BD401B4014501DAA0
:10217600000B0224023D0256025E00BA0016013030
:062186002E382E3000008F
:00000001FF
